:020000040800F2
:100000000006022001020008F50E0008F90E0008A3
:10001000510F0008F90E0008250F00080302000820
:10002000030200080302000803020008D9280008A0
:10003000030200080302000803020008030200088C
:10004000030200080302000803020008030200087C
:1000500003020008030200083D3A0008653A000860
:100060008D3A0008B53A0008DD3A0008030200089E
:10007000030200080302000803020008030200084C
:10008000030200080302000803020008030200083C
:10009000030200080302000803020008053B0008F1
:1000A000030200080302000803020008030200081C
:1000B000293C0008030200080302000803020008AC
:1000C00003020008030200080302000803020008FC
:1000D0000302000803020008D93B0008ED3B0008BA
:1000E000693B00080302000803020008030200083D
:1000F00003020008030200080302000803020008CC
:1001000003020008030200080302000803020008BB
:1001100003020008013C0008030200080302000873
:10012000030200080302000803020008030200089B
:10013000030200080302000803020008030200088B
:100140000302000803020008030200088D300008C3
:10015000030200080302000803020008030200086B
:10016000030200080302000803020008030200085B
:10017000030200080302000803020008030200084B
:100180000302000803020008153C000803020008EF
:10019000030200080302000803020008030200082B
:1001A000030200080302000803020008030200081B
:1001B000030200080302000803020008030200080B
:1001C00003020008030200080302000803020008FB
:1001D00003020008030200080302000803020008EB
:1001E00003020008030200080302000803020008DB
:1001F00003020008030200080302000803020008CB
:1002000002E000F000F8FEE772B63A4880F3088892
:10021000394880F3098839484EF60851CEF200017A
:10022000086040F20000CCF200004EF63471CEF2CD
:1002300000010860BFF34F8FBFF36F8F40F20000E3
:10024000C0F2F0004EF68851CEF200010860BFF314
:100250004F8FBFF36F8F4FF00000E1EE100A4EF6A4
:100260003C71CEF200010860062080F31488BFF3D1
:100270006F8F02F0EFFB02F091FB03F081FA4FF079
:1002800055301F491B4A91423CBF41F8040BFAE725
:100290001C49194A91423CBF41F8040BFAE71A493C
:1002A0001A4A1B4B9A423EBF51F8040B42F8040B0A
:1002B000F8E700201749184A91423CBF41F8040B67
:1002C000FAE702F0A9FB03F0BBFA144C144DAC4260
:1002D00003DA54F8041B8847F9E700F041F8114CA1
:1002E000114DAC4203DA54F8041B8847F9E702F0D9
:1002F00091BB00000006022000220220000000083E
:1003000000000220000602207040000800220220A7
:100310006822022068220220BC3B02200002000862
:100320000002000800020008000200082DE9F04F5A
:100330002DED108AC1F80CD0D0F80CD0BDEC108A8D
:10034000BDE8F08F002383F311882846A0470020E2
:1003500001F0E2FEFEE701F077FE00DFFEE70000BD
:1003600038B500F0BBFC40B1174B6FF07F010022A5
:1003700059720F211A729972DA7202F06FFA0546F9
:1003800002F0A4FA0446D0B9104B9D4219D00133B3
:100390009D4241F2883512BF044600250124002009
:1003A00002F066FA0CB100F059F800F045FD00F0DB
:1003B000D5FB284600F0E0F800F050F8F9E70025FA
:1003C000EDE70546EBE700BF00220220010007B081
:1003D00008B500F08FFBA0F120035842584108BD3A
:1003E00007B541F21203022101A8ADF8043000F074
:1003F0009FFB03B05DF804FB202310B583F3118845
:100400001248C3680BB101F00DFF0023104A4FF4EE
:100410007A710E4801F0CAFE002383F311880D4C57
:10042000236813B12368013B2360636813B16368D9
:10043000013B6360084B1B7833B9636823B9022022
:1004400000F06CFC3223636010BD00BF6822022004
:10045000F9030008842302207C220220F8B5404BD7
:10046000404A1C461968013179D004339342F9D1CE
:100470006268A24273D33C4B9B6803F1006303F5AF
:1004800000439A426BD2002000F082FB0220374BDF
:10049000187000F035FC364B00211A6C19641A6E86
:1004A00019661A6E5A6C59645A6E59665A6E5A69B0
:1004B00042F080025A615A6922F080025A615A69F8
:1004C0001A6942F000521A611A6922F000521A6148
:1004D0001B6972B64FF0E023C3F8084DD4E900045D
:1004E000BFF34F8FBFF36F8F224AC2F88410BFF360
:1004F0004F8F536923F480335361BFF34F8FD2F88A
:10050000803043F6E076C3F3C905C3F34E335B0195
:1005100003EA060C29464CEA81770139C2F8747265
:10052000F9D2203B13F1200FF2D1BFF34F8FBFF36D
:100530006F8FBFF34F8FBFF36F8F536923F4003377
:1005400053610023C2F85032BFF34F8FBFF36F8F58
:10055000202383F31188854680F308882047F8BD5F
:100560000080000820800008002202207C22022057
:100570000038024000ED00E02DE9F04F93B0A94BA8
:100580002022FF2100900AA89D6800F0FFFBA64AE8
:100590001378A3B90121A5481170C360202383F308
:1005A0001188C3680BB101F03DFE0023A04A4FF44F
:1005B0007A719E4801F0FAFD002383F31188009BB5
:1005C0009C4A03B1136000239B49009C98469B46BC
:1005D0001E469A460B705360012000F091FB24B137
:1005E000944B1B68002B00F01682002000F082FA6A
:1005F0000390039B002BF2DB012000F071FB039BB7
:10060000213B162BE8D801A252F823F06906000816
:100610009106000825070008D9050008D90500083B
:10062000D9050008B90700088B090008A5080008CB
:10063000070900082F09000855090008D905000816
:1006400067090008D9050008D9090008090700084A
:10065000D90500081D0A00087506000809070008EA
:10066000D9050008070900080220FFF7B1FE00289D
:1006700040F0FB81009B022105A8B8F1000F08BFE4
:100680001C4641F21233ADF8143000F051FAA3E7E2
:100690004FF47A7000F02EFA071EEBDB0220FFF712
:1006A00097FE0028E6D0013F052F00F2E081DFE849
:1006B00007F0030A0D1013360523042105A805933E
:1006C00000F036FA17E004215648F9E704215B48A8
:1006D000F6E704215A48F3E74FF01C09484609F1B0
:1006E000040900F057FA0421059005A800F020FA4B
:1006F000B9F12C0FF2D101204FF0000A00FA07F7F0
:1007000047EA0B0B5FFA8BFB00F08CFB26B10BF07A
:100710000B030B2B08BF0024FFF762FE5CE70421EC
:100720004848CDE7002EA5D00BF00B030B2BA1D131
:100730000220FFF74DFE074600289BD001203E4EC9
:1007400000F026FA4FF000080220307000F0D8FACE
:100750005FFA88F9484600F02BFA044690B1484603
:1007600008F1010800F034FA0028F1D1B846044637
:1007700041F21213022105A83E46ADF8143000F0F4
:10078000D7F929E7012325460220337000F0A8FAA3
:10079000244B9B68AB4207D9284600F0FBF9013097
:1007A00040F068810435F3E70025234BB8463E4608
:1007B0001D70204B5D60A7E7002E3FF45BAF0BF090
:1007C0000B030B2B7FF456AF02201B4B187000F06D
:1007D00097FA322000F08EF9B0F10009FFF64AAF27
:1007E00019F003077FF446AF0E4A09EB0503926840
:1007F00093423FF63FAFB9F5807F3FF73BAF124BD7
:10080000B945019322DD4FF47A7000F073F903903B
:10081000039A002AFFF62EAF039A0137019B03F8D3
:10082000012BEDE700220220802302206822022013
:10083000F9030008842302207C22022004220220E3
:10084000082202200C22022080220220C820FFF76A
:10085000BFFD074600283FF40DAF1F2D11D8C5F18D
:1008600020020AAB25F0030084494A45184428BFFA
:100870004A46019200F064FA019AFF217F4800F095
:1008800085FA4FEAA903C9F387027C4928460193F8
:1008900000F084FA064600283FF46AAF019B05EB9E
:1008A000830531E70220FFF793FD00283FF4E2AE15
:1008B00000F0B8F900283FF4DDAE0027B946704BD0
:1008C0009B68BB4218D91F2F11D80A9B01330ED049
:1008D00027F0030312AA134453F8203C059348461B
:1008E000042205A9043700F047FB8146E7E73846B4
:1008F00000F050F90590F2E7CDF81490042105A816
:1009000000F016F900E70023642104A8049300F026
:1009100005F900287FF4AEAE0220FFF759FD00284C
:100920003FF4A8AE049800F065F90590E6E70023CF
:10093000642104A8049300F0F1F800287FF49AAE33
:100940000220FFF745FD00283FF494AE049800F024
:1009500061F9EAE70220FFF73BFD00283FF48AAE89
:1009600000F070F9E1E70220FFF732FD00283FF4C4
:1009700081AE05A9142000F06BF90746042104900C
:1009800004A800F0D5F83946B9E7322000F0B2F8F3
:10099000071EFFF66FAEBB077FF46CAE384A07EB5D
:1009A0000A03926893423FF665AE0220FFF710FDFE
:1009B00000283FF45FAE27F003075744BA453FF4E1
:1009C000A3AE50460AF1040A00F0E4F804210590B1
:1009D00005A800F0ADF8F1E74FF47A70FFF7F8FCE6
:1009E00000283FF447AE00F01DF9002844D00A9BD0
:1009F00001330BD008220AA9002000F0CFF900280B
:100A00003AD02022FF210AA800F0C0F9FFF7E8FC45
:100A10001C4801F087FB13B0BDE8F08F002E3FF4B7
:100A200029AE0BF00B030B2B7FF424AE00236421C3
:100A300005A8059300F072F8074600287FF41AAE67
:100A40000220FFF7C5FC814600283FF413AEFFF7F4
:100A5000C7FC41F2883001F065FB059800F02AFAE6
:100A60004E463C4600F0DEF9B6E506464CE64FF051
:100A7000000AFFE5B8467BE6374679E68022022089
:100A800000220220A08601002DE9F84F4FF47A736E
:100A900006460D46002402FB03F7DFF85080DFF81E
:100AA000509098F900305FFA84FA5A1C01D0A342A2
:100AB00010D159F824002A4631460368D3F820B0F3
:100AC0003B46D847854205D1074B012083F800A05B
:100AD000BDE8F88F0134052CE3D14FF4FA7001F032
:100AE00021FB0020F4E700BFD023022010220220C7
:100AF0001C3D0008002307B5024601210DF1070047
:100B00008DF80730FFF7C0FF20B19DF8070003B054
:100B10005DF804FB4FF0FF30F9E700000A460421BE
:100B200008B5FFF7B1FF80F00100C0B2404208BD38
:100B3000074B0A4630B41978064B53F8214001465A
:100B400023682046DD69044BAC4630BC604700BFDB
:100B5000D02302201C3D0008A086010070B50A4E7B
:100B600000240A4D01F080FD3080286833888342DC
:100B700008D901F073FD2B6804440133B4F5004F2C
:100B80002B60F2D370BD00BFD22302208C23022041
:100B900001F018BE00F1006000F5004000687047E9
:100BA00000F10060920000F5004001F0A3BD0000DC
:100BB000054B1A68054B1B889B1A834202D91044C7
:100BC00001F04CBD002070478C230220D22302206C
:100BD00038B5074D04462868204401F047FD28B980
:100BE00028682044BDE8384001F058BD38BD00BF3A
:100BF0008C23022010F0030309D1B0F5846F04D2D6
:100C000000F10050A0F571200368184670470023DA
:100C1000FBE7000000F10050A0F57120D0F820049F
:100C200070470000064991F8243033B100230822B0
:100C3000086A81F82430FFF7B3BF0120704700BF76
:100C400090230220014B1868704700BF002004E089
:100C5000204B0246F0B518681F4BC0F30B06000C82
:100C60001F885D68BE4293F9084022D09F89BE422A
:100C700021D01F8BBE4206D102240C2505FB043374
:100C80005D6893F90840B0F5805F16D041F201032A
:100C9000984208BF5A24013A013D0B460A44934248
:100CA0000DD215F9016F581C5EB1034600F8016CB6
:100CB000F5E70024E1E70124DFE74124EBE71846EC
:100CC00005E02C2590421D7001D2981C5C70401AE2
:100CD000F0BD00BF002004E0142202200020704775
:100CE000022804D1054B4FF400129A617047012885
:100CF000FCD1024B4FF40022F7E700BF0010024086
:100D0000022803D1044B20229A6170470128FCD1AC
:100D1000014B0822F8E700BF00100240022805D16D
:100D2000064A536983F02003536170470128FCD1C0
:100D3000024A536983F00803F6E700BF001002403F
:100D4000002310B5934203D0CC5CC4540133F9E7BF
:100D500010BD0000013810B510F9013F3BB191F909
:100D600000409C4203D11AB10131013AF4E71AB1B3
:100D700091F90020981A10BD1046FCE70346024680
:100D8000D01A12F9011B0029FAD170470244034618
:100D9000934202D003F8011BFAE770472DE9F843AC
:100DA0001F4D14460746884695F8242052BBDFF8AD
:100DB00070909CB395F824302BB92022FF2148462F
:100DC0002F62FFF7E3FF95F824004146C0F10802C7
:100DD00005EB8000A24228BF2246D6B29200FFF760
:100DE000AFFF95F82430A41B17441E449044E4B28E
:100DF000F6B2082E85F82460DBD1FFF713FF002838
:100E0000D7D108E02B6A03EB82038342CFD0FFF7F0
:100E100009FF0028CBD10020BDE8F8830120FBE7C3
:100E200090230220024B1A78024B1A70704700BFC1
:100E3000D023022010220220F8B5184C184800F0E8
:100E4000A3FC2146164800F0CBFC24681548E26E4E
:100E5000154ED2F80438154D43F00203104FC2F876
:100E6000043801F05FF92046114900F0C1FDE26E3F
:100E70000524D2F8043823F00203C2F804384FF4F2
:100E8000E133336055F8040BB84202D0314600F02C
:100E9000DBFB013C14F0FF04F4D1F8BD303E000848
:100EA000402F022040420F00B82302201C3D0008C2
:100EB000383E000838B50B4B04461A780A4B53F8F5
:100EC00022500A4B9D420CD0094B00211822184693
:100ED000FFF75CFF046001462846BDE8384000F09B
:100EE000B3BB38BDD02302201C3D0008402F022098
:100EF000B8230220FEE7000000B59BB0EFF30981A4
:100F000068226846FFF71CFFEFF30583044B9A6BDA
:100F1000DA6A9A6A9A6A9A6A9A6A9A6A9B6AFEE78F
:100F200000ED00E000B59BB0EFF309816822684650
:100F3000FFF706FFEFF30583044B9A6B9A6A9A6AF0
:100F40009A6A9A6A9A6A9B6AFEE700BF00ED00E01F
:100F500000B59BB0EFF3098168226846FFF7F0FE09
:100F6000EFF30583034B5A6B9A6A9A6A9A6A9A6AF4
:100F70009B6AFEE700ED00E030B50A44084D91425F
:100F80000DD011F8013B5840082340F30004013B09
:100F90002C4013F0FF0384EA5000F6D1EFE730BD98
:100FA0002083B8ED026843681143016003B118471C
:100FB00070470000024A136843F0C0031360704793
:100FC00000440040024A136843F0C00313607047B6
:100FD00000480040024A136843F0C00313607047A2
:100FE00000500040024A136843F0C003136070478A
:100FF0000078004037B5334C334D204600F018FBE5
:1010000004F11400009400234FF480722F4900F083
:10101000D9F94FF480722E4904F1380000942D4B19
:1010200000F052FA2C4BC4E917352C4C204600F046
:10103000FFFA04F11400009400234FF48072284951
:1010400000F0C0F94FF48072264904F13800009492
:10105000254B00F039FA254BC4E91735244C2046BE
:1010600000F0E6FA04F11400009400234FF48072BB
:10107000204900F0A7F94FF480721F4904F13800AD
:1010800000941E4B00F020FA1D4BC4E917351D4C8F
:10109000204600F0CDFA04F1140000234FF48072D2
:1010A0001949009400F08EF9184B4FF480721849DA
:1010B00004F13800009400F007FA164BC4E9173524
:1010C00003B030BDD423022080F9370384250220E9
:1010D00084290220B50F000800440040402402206B
:1010E00084260220842A0220C50F00080048004000
:1010F000AC24022084270220842B0220D50F000874
:10110000005000401825022084280220E50F000826
:10111000842C022000780040037C30B5344C002938
:1011200018BF0C46012B16D1324B98420AD1324BD4
:101130001A6C42F400321A641A6E42F400321A66D3
:101140001B6E08E02D4B984232D02D4B984238D080
:101150002C4B98423ED02268036EC16D03EB5203C4
:101160008466B3FBF2F36268150442BF23F00705FF
:1011700003F0070343EA4503CB60A36843F0400351
:101180004B60E36843F001038B6042F4967343F0D5
:1011900001030B604FF0FF330B62510505D512F0D0
:1011A000102220D0B2F1805F1FD080F8643030BDB3
:1011B000114B1A6C42F480221A641A6E42F4802297
:1011C000BDE70D4B1A6C42F480121A641A6E42F499
:1011D0008012B4E7084B1A6C42F080421A641A6E0F
:1011E00042F08042ABE77F23DFE73F23DDE700BF2C
:1011F000303D0008D4230220003802404024022061
:10120000AC240220182502202DE9F047C66D0546C2
:101210003768F4692107346219D014F0080118BF47
:101220008021E20748BF41F02001A3074FF02003CF
:1012300048BF41F04001600748BF41F4807183F32B
:101240001188281DFFF7AEFE002383F31188E20505
:101250000AD5202383F311884FF40071281DFFF76E
:10126000A1FE002383F311884FF020094FF0000AFC
:1012700014F0200838D13B0616D54FF0200905F1AF
:10128000380A200610D589F31188504600F050F92D
:10129000002836DA0821281DFFF784FE27F0800396
:1012A0003360002383F31188790614D5620612D5C2
:1012B000202383F31188D5E913239A4208D12B6C9C
:1012C00033B127F040071021281DFFF76BFE376070
:1012D000002383F31188E30618D5AA6E1369ABB116
:1012E0005069BDE8F047184789F31188736A2846AA
:1012F00095F86410194000F0B5F98AF31188F46983
:10130000B6E7B06288F31188F469BAE7BDE8F08700
:10131000F8B51546826804460B46AA4200D2856895
:10132000A1692669761AB5420BD218462A46FFF7FC
:1013300007FDA3692B44A3612846A3685B1BA36038
:10134000F8BD0CD9AF1B18463246FFF7F9FC3A46F8
:10135000E1683044FFF7F4FCE3683B44EBE71846F0
:101360002A46FFF7EDFCE368E5E700008368934257
:10137000F7B50446154600D28568D4E90460361AEC
:10138000B5420BD22A46FFF7DBFC63692B4463614D
:101390002846A3685B1BA36003B0F0BD0DD932469D
:1013A000AF1B0191FFF7CCFC01993A46E06831444C
:1013B000FFF7C6FCE3683B44E9E72A46FFF7C0FCB9
:1013C000E368E4E710B50A440024C361029B84602B
:1013D000C16002610362C0E90000C0E9051110BDEF
:1013E00008B5D0E90532934201D1826882B982689A
:1013F000013282605A1C426119700021D0E9043226
:101400009A4224BFC368436100F0A8FE002008BDD3
:101410004FF0FF30FBE7000070B5202304460E4676
:1014200083F31188A568A5B1A368A269013BA360F5
:10143000531CA36115782269934224BFE368A3611A
:10144000E3690BB120469847002383F311882846AF
:1014500007E03146204600F071FE0028E2DA85F30D
:10146000118870BD2DE9F74F04460E461746984681
:10147000D0F81C904FF0200A8AF311884FF0000B2F
:10148000154665B12A4631462046FFF741FF03461F
:1014900060B94146204600F051FE0028F1D00023FB
:1014A00083F31188781B03B0BDE8F08FB9F1000F0A
:1014B00003D001902046C847019B8BF31188ED1A99
:1014C0001E448AF31188DCE7C160C361009B82601F
:1014D0000362C0E905111144C0E9000001617047D1
:1014E000F8B504460D461646202383F31188A768F5
:1014F000A7B1A368013BA36063695A1C62611D70B8
:10150000D4E904329A4224BFE3686361E3690BB112
:1015100020469847002080F3118807E03146204696
:1015200000F00CFE0028E2DA87F31188F8BD000015
:10153000D0E9052310B59A4201D182687AB9826850
:101540000021013282605A1C82611C7803699A4230
:1015500024BFC368836100F001FE204610BD4FF038
:10156000FF30FBE72DE9F74F04460E461746984635
:10157000D0F81C904FF0200A8AF311884FF0000B2E
:10158000154665B12A4631462046FFF7EFFE034671
:1015900060B94146204600F0D1FD0028F1D000237B
:1015A00083F31188781B03B0BDE8F08FB9F1000F09
:1015B00003D001902046C847019B8BF31188ED1A98
:1015C0001E448AF31188DCE7026843681143016016
:1015D00003B11847704700001430FFF743BF000005
:1015E0004FF0FF331430FFF73DBF00003830FFF7F6
:1015F000B9BF00004FF0FF333830FFF7B3BF000032
:101600001430FFF709BF00004FF0FF311430FFF72F
:1016100003BF00003830FFF763BF00004FF0FF3218
:101620003830FFF75DBF000000207047FFF7E2BCD5
:10163000044B036000234360C0E9023301230374B9
:10164000704700BF483D000810B52023044683F3CF
:101650001188FFF761FD02232374002383F31188AF
:1016600010BD000038B5C36904460D461BB90421FE
:101670000844FFF7A9FF294604F11400FFF7B0FE64
:10168000002806DA201D4FF48061BDE83840FFF7DE
:101690009BBF38BD026843681143016003B118471E
:1016A0007047000013B5446BD4F8A4381A68117859
:1016B000042915D1217C022912D11979012312891B
:1016C0008B4013420CD101A904F14C0001F05EFFE4
:1016D000D4F8A4480246019B2179206800F0D4F98F
:1016E00002B010BD143001F0E1BE00004FF0FF3336
:1016F000143001F0DBBE00004C3001F0B3BF00003D
:101700004FF0FF334C3001F0ADBF0000143001F05A
:10171000AFBE00004FF0FF31143001F0A9BE000051
:101720004C3001F07FBF00004FF0FF324C3001F031
:1017300079BF000000207047D0F8A4381A6810B5AF
:1017400011780446042917D1017C022914D1597952
:10175000012352898B4013420ED1143001F042FE16
:10176000024648B1D4F8A4484FF4807361792068E8
:10177000BDE8104000F076B910BD0000406BFFF7E7
:10178000DBBF0000704700007FB5124B0125042627
:10179000044603600023057400F184024360294677
:1017A000C0E902330C4B0290143001934FF4807364
:1017B000009601F0F3FD094B04F29442294604F12E
:1017C0004C000294CDE900634FF4807301F0BAFE3F
:1017D00004B070BD703D00087D170008A516000814
:1017E0000B68202282F311880A7903EB82021062CF
:1017F0004A790D3243F822008A7912B103EB820351
:1018000018620223C0F8A4180374002383F311881C
:101810007047000038B5037F044613B190F8543088
:10182000ABB90125201D0221FFF734FF04F114009C
:101830006FF00101257700F09DFC04F14C0084F865
:1018400054506FF00101BDE8384000F093BC38BD42
:1018500010B5012104460430FFF71CFF0023237755
:1018600084F8543010BD000038B50446002514300B
:1018700001F0ACFD04F14C00257701F07BFE201D4A
:1018800084F854500121FFF705FF2046BDE8384099
:10189000FFF752BF90F85C3003F06003202B06D1B5
:1018A00090F85D200023212A03D81F2A06D80020A3
:1018B0007047222AFBD1C0E9143303E0034A0265D2
:1018C0000722426583650120704700BF382202204D
:1018D000D0F8A43837B51A680446117804291AD10B
:1018E000017C022917D11979012312898B401342F7
:1018F00011D100F14C05284601F0FCFE58B101A9B8
:10190000284601F043FED4F8A4480246019B217901
:10191000206800F0B9F803B030BD000000EB81038F
:10192000F0B51E6A85B004460D46FEB1202383F350
:10193000118804EB8507301D0821FFF7ABFEFB681B
:1019400006F14C005B691B681BB1019001F02CFE95
:10195000019803A901F01AFE024648B1039B2946EB
:10196000204600F091F8002383F3118805B0F0BD04
:10197000FB685A691268002AF5D01B8A013B1340A4
:10198000F1D104F15C02EAE70D3138B550F821409D
:10199000DCB1202383F31188D4F8A428136852798A
:1019A00003EB8203DB689B695D6845B10421601825
:1019B000FFF770FE294604F1140001F01DFD2046DA
:1019C000FFF7BAFE002383F3118838BD704700008B
:1019D00001F0B6B801232822002110B5044600F812
:1019E000243BFFF7D3F90023C4E9013310BD000005
:1019F00038B50446202383F3118800254160C0E9EF
:101A00000355C0E90555C0E9075501F0A9F80223BF
:101A1000237085F3118838BD70B500EB810305464E
:101A200050690E461446DA6018B110220021FFF703
:101A3000ADF9A06918B110220021FFF7A7F93146CE
:101A40002846BDE8704001F055B90000826802F0F8
:101A5000011282600022C0E90422C0E9062202626B
:101A600001F0D4B9F0B4012500EB810447898D4021
:101A7000E4683D43A469458123600023A26063605C
:101A8000F0BC01F0EFB90000F0B4012500EB8104D7
:101A900007898D40E4683D43646905812360002324
:101AA000A2606360F0BC01F069BA000070B5022367
:101AB0000025044603704566056280F84C50C0E975
:101AC0000255C0E90455C0E9065501F0AFF8636856
:101AD0001B6823B129462046BDE87040184770BDF9
:101AE000037880F868300523037043681B6810B5DD
:101AF00004460BB1042198470023A36010BD0000E9
:101B000090F86820436802701B680BB105211847E4
:101B10007047000070B590F84C30044613B10023B4
:101B200080F84C3004F15C02204601F091F96368C2
:101B30009B68B3B994F85C3013F0600535D0002190
:101B4000204601F0F7FB0021204601F0E9FB636825
:101B50001B6813B1062120469847062384F84C30B1
:101B600070BD204698470028E4D0B4F86230626D1A
:101B70009A4288BF636594F95C30656D002B4FF025
:101B8000200380F20381002D00F0F280092284F806
:101B90004C2083F3118800212046D4E91423FFF759
:101BA00073FF002383F31188DAE794F85D2003F0D4
:101BB0007F0343EA022340F20232934200F0C580E1
:101BC00021D8B3F5807F48D00DD8012B3FD0022B10
:101BD00000F09380002BB2D104F16402226502224E
:101BE0006265A365C1E7B3F5817F00F09B80B3F523
:101BF000407FA4D194F85E30012BA0D1B4F86430BA
:101C000043F0020332E0B3F5006F4DD017D8B3F5BF
:101C1000A06F31D0A3F5C063012B90D86368204634
:101C200094F85E205E6894F85F10B4F86030B047B6
:101C3000002884D043682365036863651AE0B3F520
:101C4000106F36D040F6024293427FF478AF5C4B7F
:101C50002365022363650023C3E794F85E30012BFC
:101C60007FF46DAFB4F8643023F00203A4F864305D
:101C7000C4E91455A56578E7B4F85C30B3F5A06FF6
:101C80000ED194F85E30204684F8663001F026F8D4
:101C900063681B6813B10121204698470323237012
:101CA0000023C4E914339CE704F16703236501238F
:101CB000C3E72378042B10D1202383F31188204617
:101CC000FFF7C4FE85F311880321636884F8675029
:101CD00021701B680BB12046984794F85E30002BAA
:101CE000DED084F867300423237063681B68002B00
:101CF000D6D0022120469847D2E794F8603020469B
:101D00001D0603F00F010AD501F094F8012804D054
:101D100002287FF414AF2B4B9AE72B4B98E701F086
:101D20007BF8F3E794F85E30002B7FF408AF94F86B
:101D3000603013F00F01B3D01A06204602D501F02F
:101D40000DFBADE701F000FBAAE794F85E30002B35
:101D50007FF4F5AE94F8603013F00F01A0D01B06AD
:101D6000204602D501F0E6FA9AE701F0D9FA97E7A2
:101D7000142284F84C2083F311882B462A462946E6
:101D80002046FFF76FFE85F31188E9E65DB1152265
:101D900084F84C2083F3118800212046D4E91423D1
:101DA000FFF760FEFDE60B2284F84C2083F31188D8
:101DB0002B462A4629462046FFF766FEE3E700BF8A
:101DC000A03D0008983D00089C3D000838B590F8FB
:101DD0004C300446002B3ED0063BDAB20F2A34D8F2
:101DE0000F2B32D8DFE803F037313108223231319E
:101DF0003131313131313737456DB0F862309D4284
:101E000014D2C3681B8AB5FBF3F203FB12556DB9FC
:101E1000202383F311882B462A462946FFF734FEF8
:101E200085F311880A2384F84C300EE0142384F8DB
:101E30004C30202383F31188002320461A4619468C
:101E4000FFF710FE002383F3118838BD836D03B1C3
:101E500098470023E7E70021204601F06BFA0021B4
:101E6000204601F05DFA63681B6813B10621204625
:101E700098470623D7E7000010B590F84C30044689
:101E8000142B29D017D8062B05D001D81BB110BDB3
:101E9000093B022BFBD80021204601F04BFA002120
:101EA000204601F03DFA63681B6813B10621204605
:101EB0009847062319E0152BE9D10B2380F84C3005
:101EC000202383F3118800231A461946FFF7DCFD0F
:101ED000002383F31188DAE7C3689B695B68002BF2
:101EE000D5D1836D03B19847002384F84C30CEE7F9
:101EF000024B0022C3E900339A607047842D022010
:101F0000002382680374054B1B6899689142FBD2D9
:101F10005A6803604260106058607047842D022048
:101F200008B5202383F31188037C032B05D0042BF1
:101F30000DD02BB983F3118808BD436900221A60C4
:101F40004FF0FF334361FFF7DBFF0023F2E7D0E9F7
:101F5000003213605A60F3E7002382680374054B74
:101F60001B6899689142FBD85A6803604260106010
:101F700058607047842D0220054B19690874186851
:101F8000026853601A60186101230374FEF7CEB92A
:101F9000842D02204B1C30B5044687B00A4D10D06A
:101FA0002B6901A8094A00F001F92046FFF7E4FF78
:101FB000049B13B101A800F035F92B69586907B0EB
:101FC00030BDFFF7D9FFF8E7842D0220211F00085C
:101FD00038B50C4D044641612B6981689A6891427D
:101FE00003D8BDE83840FFF78BBF1846FFF7B4FFB2
:101FF00001232C61014623742046BDE83840FEF7DA
:1020000095B900BF842D0220044B1A681B699068A3
:102010009B68984294BF002001207047842D0220C5
:1020200010B5084C236820691A68546022600122A8
:1020300023611A74FFF790FF01462069BDE8104044
:10204000FEF774B9842D0220FFF7EABFFEE7000017
:1020500010B50C4CFFF74CFF00F09AF880220A49AB
:10206000204600F021F8012344F8180C037400F016
:1020700043FC002383F3118862B60448BDE8104096
:1020800000F032B8AC2D0220A43D0008B43D000899
:1020900000F002B9034A516853685B1A9842FBD8B2
:1020A000704700BF001000E0826002220282704789
:1020B0008368A3F17C0243F80C2C026943F83C2CA2
:1020C000426943F8382C074A43F81C2CC268A3F134
:1020D000180043F8102C022203F8082C002203F801
:1020E000072C70474503000810B5202383F311889F
:1020F000FFF7DEFF00210446FFF76AFF002383F3AA
:102100001188204610BD0000024B1B6958610F204A
:10211000FFF732BF842D0220202383F31188FFF7BD
:10212000F3BF000008B50146202383F3118808207F
:10213000FFF730FF002383F3118808BD49B1064B38
:1021400042681B6918605A60136043600420FFF7FF
:1021500021BF4FF0FF307047842D02200368984262
:1021600006D01A680260506018465961FFF7C8BE71
:102170007047000038B504460D462068844200D1FF
:1021800038BD036823605C604561FFF7B9FEF4E782
:10219000054B4FF0FF3103F11402C3E90522002281
:1021A000C3E90712704700BF842D022070B51C4E92
:1021B00005460C46C0E9032301F0CEFA334653F836
:1021C000142F9A420DD130620A2C2CBF00190A300C
:1021D0002A60C5E90124C6E90555BDE8704001F053
:1021E000A9BA316A431AE31838BF1C469368A34260
:1021F00002D9081901F0ACFA73699A6894420CD8B4
:102200005A68AC602B606A6015609A685D60121B4A
:102210009A604FF0FF33F36170BDA41A1B68ECE7BE
:10222000842D022038B51B4C636998420DD081681B
:10223000D0E9003213605A600022C2609A680A44F2
:102240009A604FF0FF33E36138BD036822460021F6
:1022500042F8143F93425A60C16003D1BDE8384050
:1022600001F070BA9A688168256A0A449A6001F0A0
:1022700073FA6369411B9A688A42E5D9AB181D1A43
:10228000206A092D98BF01F10A02BDE838401044C8
:1022900001F05EBA842D02202DE9F041184C002790
:1022A00004F11406656901F057FA236AAA68C11A95
:1022B0008A4215D81344D5F80C802362D5E9003240
:1022C00013605A606369EF60B34201D101F03AFADA
:1022D00087F311882869C047202383F31188E1E739
:1022E0006169B14209D013441B1ABDE8F0410A2BC1
:1022F0002CBFC0180A3001F02BBABDE8F08100BF36
:10230000842D022000207047FEE700007047000087
:102310004FF0FF307047000002290CD0032904D091
:102320000129074818BF00207047032A05D805482F
:1023300000EBC2007047044870470020704700BFA0
:10234000943E000848220220483E000870B59AB02A
:1023500005460846144601A900F0C2F801A8FEF798
:102360000DFD431C0022C6B25B001046C5E90034D7
:1023700023700323023404F8013C01ABD1B20234D0
:102380008E4201D81AB070BD13F8011B013204F857
:10239000010C04F8021CF1E708B5202383F311882F
:1023A0000348FFF795FA002383F3118808BD00BFA7
:1023B000402F022090F85C3003F01F02012A07D161
:1023C00090F85D200B2A03D10023C0E9143315E0F7
:1023D00003F06003202B08D1B0F860302BB990F8DF
:1023E0005D20212A03D81F2A04D8FFF753BA222AD6
:1023F000EBD0FAE7034A02650722426583650120B4
:10240000704700BF3F22022007B5052917D8DFE833
:1024100001F0191603191920202383F31188104A9B
:1024200001210190FFF7F8FA019802210D4AFFF708
:10243000F3FA0D48FFF718FA002383F3118803B06D
:102440005DF804FB202383F311880748FFF7E2F9C6
:10245000F2E7202383F311880348FFF7F9F9EBE74C
:10246000E83D00080C3E0008402F022038B50C4D16
:102470000C4C2A460C4904F10800FFF767FF05F1F0
:10248000CA0204F110000949FFF760FF05F5CA729E
:1024900004F118000649BDE83840FFF757BF00BFF8
:1024A0001838022048220220CC3D0008D43D000804
:1024B000DF3D000870B5044608460D46FEF75EFC99
:1024C000C6B22046013403780BB9184670BD3246B7
:1024D0002946FEF73FFC0028F3D10120F6E7000073
:1024E0002DE9F84F05460C46FEF748FC2C49C6B2CC
:1024F0002846FFF7DFFF08B10236F6B22949284621
:10250000FFF7D8FF08B11036F6B2632E0DD8DFF80A
:102510009080DFF89090244FDFF894A0DFF894B01B
:102520002E7846B92670BDE8F88F29462046BDE8CA
:10253000F84F01F0D5BB252E2ED107224146284663
:10254000FEF708FC70B9DBF800300735093444F8B1
:10255000093CDBF8043044F8053C9BF8083004F8EB
:10256000013CDDE7082249462846FEF7F3FB98B90F
:10257000A21C0E4B197802320909C95D02F8041C2D
:1025800013F8011B01F00F015345C95D02F8031C4C
:10259000F0D118340835C3E7013504F8016BBFE703
:1025A000B43E0008DF3D0008C63E000820F4F01FDE
:1025B0002CF4F01FBC3E0008BFF34F8F024AD368D3
:1025C000DB03FCD4704700BF003C024008B5074B5A
:1025D0001B7853B9FFF7F0FF054B1A69002A04DA9C
:1025E000044A5A6002F188325A6008BD763A0220E5
:1025F000003C02402301674508B5054B1B7833B901
:10260000FFF7DAFF034A136943F00043136108BD83
:10261000763A0220003C02400B28F0B516D80C4C4C
:102620000C4923787BB90E460B4D0C234FF000620A
:10263000013B55F8047B46F8042B13F0FF033A44A2
:10264000F6D10123237051F82000F0BD0020FCE7F3
:10265000A83A0220783A0220D83E0008014B53F8ED
:1026600020007047D83E00080C2070470B2810B59A
:10267000044601D9002010BDFFF7CEFF064B53F8EA
:1026800024301844C21A0BB90120F4E71268013251
:10269000F0D1043BF6E700BFD83E00080B2810B588
:1026A000044621D8FFF788FFFFF790FF0F4AF32376
:1026B000D360C300DBB243F4007343F00203136141
:1026C000136943F480331361FFF776FFFFF7A4FF2C
:1026D000074B53F8241000F0D9F82046FFF78CFF81
:1026E000BDE81040FFF7C2BF002010BD003C024013
:1026F000D83E0008F8B512F00103144642D1821802
:10270000B2F1026F57D22D4B1B6813F0010352D068
:10271000FFF75CFF2A4DF32340F20127EB60FFF740
:102720004BFF032C15D824F00104401A40F2011786
:102730006618234CB14200EB0105236924D123F034
:10274000010301202361FFF757FFF8BD043C04306B
:10275000E7E78307E7D12B6923F440732B612B69EB
:102760003B432B6151F8046B0660BFF34F8FFFF7BB
:1027700023FF03689E42E9D02B6923F001032B61FC
:10278000FFF73AFF0020E0E723F440732361236959
:102790003B4323610B882B80BFF34F8FFFF70CFF68
:1027A0002D88ADB231F8023BAB42C3D0236923F090
:1027B00001032361E4E71846C7E700BF0038024081
:1027C000003C0240084908B50B7828B11BB9FFF757
:1027D000FDFE01230B7008BD002BFCD00870BDE886
:1027E0000840FFF709BF00BF763A02200244074BBA
:1027F000D2B210B5904200D110BD441C00B253F8C3
:10280000200041F8040BE0B2F4E700BF502800407C
:102810000F4B30B51C6F240407D41C6F44F40074B4
:102820001C671C6F44F400441C670A4C0244236874
:10283000D2B243F480732360074B904200D130BD85
:10284000441C51F8045B00B243F82050E0B2F4E7B6
:1028500000380240007000405028004007B50122B7
:1028600001A90020FFF7C2FF019803B05DF804FB47
:1028700013B50446FFF7F2FFA04205D0012201A9DB
:1028800000200194FFF7C4FF02B010BD0144BFF364
:102890004F8F064B884204D3BFF34F8FBFF36F8F28
:1028A0007047C3F85C022030F4E700BF00ED00E0A1
:1028B000044BD3F874389B0042BF034B01221A70BB
:1028C000704700BF00300240A93A0220014B18783F
:1028D000704700BFA93A0220EFF309830549683326
:1028E0004A6B22F001024A6383F30988002383F3D1
:1028F0001188704700EF00E0202080F3118862B655
:102900000D4B0E4AD96821F4E0610904090C0A4311
:102910000B49DA60D3F8FC2042F08072C3F8FC2047
:10292000084AC2F8B01F116841F00101116010227D
:10293000DA7783F82200704700ED00E00003FA0523
:1029400055CEACC5001000E0202310B583F31188EC
:102950000E4B5B6813F4006314D0F1EE103AEFF302
:1029600009844FF08073683CE361094BDB6B23669D
:1029700084F30988FFF748FB10B1064BA36110BD33
:10298000054BFBE783F31188F9E700BF00ED00E09A
:1029900000EF00E0570300085A03000870B5BFF3CA
:1029A0004F8FBFF36F8F1A4A0021C2F85012BFF346
:1029B0004F8FBFF36F8F536943F400335361BFF3FD
:1029C0004F8FBFF36F8FC2F88410BFF34F8FD2F8D1
:1029D000803043F6E074C3F3C900C3F34E335B01A8
:1029E00003EA0406014646EA81750139C2F86052DD
:1029F000F9D2203B13F1200FF2D1BFF34F8F53696F
:102A000043F480335361BFF34F8FBFF36F8F70BDBB
:102A100000ED00E0FEE700000A4B0B480B4A904235
:102A20000BD30B4BC11EDA1C121A22F003028B428D
:102A300038BF00220021FEF7A9B953F8041B40F863
:102A4000041BECE7D8400008BC3B0220BC3B022042
:102A5000BC3B02207047000070B5D0E91B43002248
:102A60004FF0FF359E6804EB42135101D3F8000983
:102A7000002805DAD3F8000940F08040C3F80009C7
:102A8000D3F8000B002805DAD3F8000B40F08040A3
:102A9000C3F8000B013263189642C3F80859C3F813
:102AA000085BE0D24FF00113C4F81C3870BD000081
:102AB0001D4B03EB8002D2F80CC02DE9F043DCF88B
:102AC0001420461CDD6ED2F800E005EB063605EB5F
:102AD0004018516871450AD30122D5F8343802FAFA
:102AE00000F023EA0000C5F83408BDE8F083AEEB3F
:102AF0000103BCF81040A34228BF2346D8F8184968
:102B0000A4B2B3EB840FF0D89468A4F1040959F887
:102B1000047F3760A4EB09071F44042FF7D81C4437
:102B20000B4494605360D4E7AC3A0220890141F031
:102B30002001016103699B06FCD41220FFF7AABAA9
:102B400010B5054C2046FEF745FF4FF0A043E36665
:102B5000024B236710BD00BFAC3A02202C3F000897
:102B600070B503780546012B50D12A4BC46E9842AC
:102B70001BD1294B0E2143205A6B42F080025A632D
:102B80005A6D42F080025A655A6D5A6942F08002CD
:102B90005A615A6922F080025A615B6900F0E8FBD1
:102BA0001E4BE3601E4BC4F800380023EE6EC4F8E1
:102BB000003EC02323604FF40413A3633369002B4A
:102BC000FCDA01230C203361FFF764FA3369DB0779
:102BD000FCD41220FFF75EFA3369002BFCDA0026E2
:102BE0002846A660FFF738FF6B68C4F81068DB68FA
:102BF000C4F81468C4F81C684BB90A4BA3614FF0C1
:102C0000FF336361A36843F00103A36070BD064B0B
:102C1000F4E700BFAC3A0220003802404014004004
:102C200003002002003C30C0083C30C0F8B5C46E40
:102C3000054600214FF000662046FFF777FF296F19
:102C400000234FF001128F684FF0FF30C4F8343882
:102C5000C4F81C2804EB431201339F42C2F80069F8
:102C6000C2F8006BC2F80809C2F8080BF2D20B6870
:102C7000EA6E6B67636210231361166916F0100623
:102C8000FBD11220FFF706FAD4F8003823F4FE63D4
:102C9000C4F80038A36943F4402343F01003A36150
:102CA0000923C4F81038C4F814380A4BEB604FF00D
:102CB000C043C4F8103B084BC4F8003BC4F810698B
:102CC000C4F800396B6F03F1100243F480136A6794
:102CD000A362F8BD083F000840800010C26E90F863
:102CE0006610D2F8003823F4FE6343EA0113C2F8F9
:102CF000003870472DE9F84300EB8103C56E0C46A0
:102D00008046DA680FFA81F94801166806F0030672
:102D1000731E022B05EB41134FF0000194BFB60464
:102D2000384EC3F8101B4FF0010104F1100398BF97
:102D300006F1805601FA03F3916998BF06F5004643
:102D400000293AD0578A04F15801374349016F509E
:102D5000D5F81C180B430021C5F81C382B18012787
:102D6000C3F81019A7405369611E9BB3138A928B55
:102D70009B08012A88BF5343D8F87420981842EA68
:102D8000034301F140022146C8F87400284605EBD0
:102D900082025360FFF7CAFE08EB8900C3681B8AF2
:102DA00043EA845348341E4364012E51D5F81C383D
:102DB0001F43C5F81C78BDE8F88305EB4917D7F821
:102DC000001B21F40041C7F8001BD5F81C1821EAAC
:102DD0000303C0E704F13F030B4A2846214605EBF5
:102DE00083035A60FFF7A2FE05EB4910D0F80039C3
:102DF00023F40043C0F80039D5F81C3823EA07074C
:102E0000D7E700BF0080001000040002026F1268C4
:102E10004267FFF721BE00005831C36E49015B587D
:102E200013F4004004D013F4001F0CBF0220012053
:102E3000704700004831C36E49015B5813F40040ED
:102E400004D013F4001F0CBF0220012070470000C3
:102E500000EB8101CB68196A0B6813604B68536003
:102E60007047000000EB810330B5DD68AA69136884
:102E7000D36019B9402B84BF402313606B8A146858
:102E8000C26E1C4402EB4110013C09B2B4FBF3F4E6
:102E90006343033323F0030343EAC44343F0C043D3
:102EA000C0F8103B2B6803F00303012B0ED1D2F8BE
:102EB000083802EB411013F4807FD0F8003B14BFB8
:102EC00043F0805343F00053C0F8003B02EB411243
:102ED000D2F8003B43F00443C2F8003B30BD000091
:102EE0002DE9F041244D0446EE6E06EB4013D3F875
:102EF000087B3807C3F8087B0AD5D6F814381907B9
:102F000006D505EB840321462846DB685B689847B5
:102F1000FA071FD5D6F81438DB071BD505EB840359
:102F2000D968CCB98B69488A5A68B2FBF0F600FBC5
:102F300016228AB91868DA6890420DD2121AC3E9CB
:102F40000024202383F311880B482146FFF78AFFD2
:102F500084F31188BDE8F081012303FA04F26B8940
:102F600023EA02036B81CB68002BF3D02146024891
:102F7000BDE8F041184700BFAC3A022000EB8103E6
:102F80004A0170B5DD68C36E6C692668E66056BBA1
:102F90001A444FF40020C2F810092A6802F0030214
:102FA000012A0AB20ED1D3F8080803EB421410F438
:102FB000807FD4F8000914BF40F0805040F00050EA
:102FC000C4F8000903EB4212D2F8000940F00440B3
:102FD000C2F800090122D3F8340802FA01F10143D2
:102FE000C3F8341870BD19B9402E84BF402020604A
:102FF00020681A442E8A8419013CB4FBF6F440EA96
:10300000C44040F00050C6E7F8B504461E48C56EFF
:1030100005EB4413D3F80869F107C3F8086917D51D
:10302000D5F81038DA0713D500EB8403D9684B695B
:103030001F68DA68974218D2D21B00271A605F60B7
:10304000202383F311882146FFF798FF87F3118827
:10305000330617D50123D5F83428A340134211D0E5
:103060002046BDE8F840FFF723BD012303FA04F230
:10307000038923EA020303818B68002BE8D02146F1
:103080009847E5E7F8BD00BFAC3A02202DE9F74FBD
:10309000A24CE66E7569B3691D4015F480587561E0
:1030A00007D02046FEF702FD03B0BDE8F04FFFF762
:1030B0004BBC002D12DAD6F8003E9F0705D0D6F89B
:1030C000003E23F00303C6F8003ED6F804389348C8
:1030D00023F00103C6F80438FEF712FD280505D5D4
:1030E0008E48FFF7B9FC8D48FEF7FAFCA9040CD511
:1030F000D6F8083813F0060FF36823F470530CBFAA
:1031000043F4105343F4A053F3602A0704D56368D3
:10311000DB680BB181489847EB0200F18A80AF026F
:1031200027D5D4F86C9000274FF0010ADFF8ECB1F6
:1031300009EB4712D2F8003B03F44023B3F5802F8C
:1031400011D1D2F8003B002B0DDA62890AFA07F39D
:1031500022EA0303638104EB8703DB68DB6813B1B6
:103160003946584698470137236FFFB29B689F4204
:10317000DED9E80618D5E76E3A6AC2F30A1002F003
:103180000F0302F4F012B2F5802F00F09C80B2F52C
:10319000402F09D104EB8303002207F58057DB6839
:1031A0001B6A904240F082802B03D6F818481DD548
:1031B000E70302D50020FFF793FEA60302D5012006
:1031C000FFF78EFE600302D50220FFF789FE210380
:1031D00002D50320FFF784FEE20202D50420FFF7A8
:1031E0007FFEA30202D50520FFF77AFE6F037FF56D
:1031F0005BAFE60702D50020FFF706FFA50702D563
:103200000120FFF701FF600702D50220FFF7FCFE57
:10321000210702D50320FFF7F7FEE20602D50420BE
:10322000FFF7F2FEA3067FF53FAF0520FFF7ECFEA8
:103230003AE7E36E00274FF0010ADFF8E0B00193B0
:10324000236F5FFA87F99B6899453FF668AF019B4A
:1032500003EB4913D3F8002902F44022B2F5802F82
:1032600022D1D3F80029002A1EDAD3F8002942F02F
:103270009042C3F80029D3F80029002AFBDB494615
:10328000E06EFFF753FC22890AFA09F322EA0303EE
:10329000238104EB8903DB689B6813B149465846D8
:1032A00098474846FFF704FC0137C9E7910701D169
:1032B000D7F80080072A02F101029CBF03F8018BB6
:1032C0004FEA18286DE7023307F5805704EB8302B5
:1032D0005268D2F818C0DCF80820DCE9001CA1EB29
:1032E0000C0C002188420AD104EB830463689B69BB
:1032F0009A6802449A605A6802445A6054E711F08E
:10330000030F01D1D7F800808C4501F1010184BF82
:1033100002F8018B4FEA1828E4E700BFAC3A02201C
:10332000C36E03EB4111D1F8003B43F40013C1F825
:10333000003B7047C36E03EB4111D1F8003943F4F1
:103340000013C1F800397047C36E03EB4111D1F887
:10335000003B23F40013C1F8003B7047C36E03EB3E
:103360004111D1F8003923F40013C1F80039704736
:10337000090100F16043012203F56143C9B283F8FA
:10338000001300F01F039A4043099B0003F16043C0
:1033900003F56143C3F880211A60704730B50433E8
:1033A000039C0172002104FB0325C160C0E90653A0
:1033B000049B0363059BC0E90000C0E90422C0E947
:1033C0000842C0E90A11436330BD00000022416A8F
:1033D000C260C0E90411C0E90A226FF00101FEF7E2
:1033E000C9BE0000D0E90432934201D1C2680AB9D3
:1033F000181D704700207047036919600021C268DA
:103400000132C260C269134482699342036124BFDE
:10341000436A0361FEF7A2BE38B504460D46E36871
:103420003BB162690020131D1268A3621344E3627A
:1034300007E0237A33B929462046FEF77FFE0028AD
:10344000EDDA38BD6FF00100FBE70000C368C26928
:10345000013BC3604369134482699342436124BFC3
:10346000436A436100238362036B03B118477047CB
:1034700070B52023044683F31188866A3EB9FFF7AE
:10348000CBFF054618B186F31188284670BDA36AA4
:10349000E26A13F8015B9342A36202D32046FFF76E
:1034A000D5FF002383F31188EFE700002DE9F84FE3
:1034B00004460E46174698464FF0200989F31188B6
:1034C0000025AA46D4F828B0BBF1000F09D1414627
:1034D0002046FFF7A1FF20B18BF311882846BDE8F5
:1034E000F88FD4E90A12A7EB050B521A934528BFAF
:1034F0009346BBF1400F1BD9334601F1400251F80E
:10350000040B914243F8040BF9D1A36A40364035CD
:103510004033A362D4E90A239A4202D32046FFF73C
:1035200095FF8AF31188BD42D8D289F31188C9E783
:1035300030465A46FDF704FCA36A5E445D445B4492
:10354000A362E7E710B5029C0433017204FB032178
:10355000C460C0E906130023C0E90A33039B036378
:10356000049BC0E90000C0E90422C0E908424363AB
:1035700010BD0000026A6FF00101C260426AC0E93A
:1035800004220022C0E90A22FEF7F4BDD0E9042398
:103590009A4201D1C26822B9184650F8043B0B6028
:1035A0007047002070470000C3680021C2690133E2
:1035B000C3604369134482699342436124BF436AF1
:1035C0004361FEF7CBBD000038B504460D46E36805
:1035D0003BB1236900201A1DA262E2691344E36231
:1035E00007E0237A33B929462046FEF7A7FD0028D5
:1035F000EDDA38BD6FF00100FBE7000003691960E8
:10360000C268013AC260C26913448269934203618D
:1036100024BF436A036100238362036B03B118472D
:103620007047000070B520230D460446114683F311
:103630001188866A2EB9FFF7C7FF10B186F311888B
:1036400070BDA36A1D70A36AE26A01339342A3624C
:1036500004D3E16920460439FFF7D0FF002080F34E
:103660001188EDE72DE9F84F04460D46904699463E
:103670004FF0200A8AF311880026B346A76A4FB993
:1036800049462046FFF7A0FF20B187F31188304656
:10369000BDE8F88FD4E90A073A1AA8EB0607974263
:1036A00028BF1746402F1BD905F1400355F8042BBE
:1036B0009D4240F8042BF9D1A36A40364033A362FF
:1036C000D4E90A239A4204D3E16920460439FFF77A
:1036D00095FF8BF311884645D9D28AF31188CDE73F
:1036E00029463A46FDF72CFBA36A3D443E443B4441
:1036F000A362E5E7D0E904239A4217D1C3689BB1DE
:10370000836A8BB1043B9B1A0ED01360C368013BE4
:10371000C360C3691A4483699A42026124BF436A41
:103720000361002383620123184670470023FBE7EF
:1037300000F094B84FF08043002258631A610222CF
:10374000DA6070474FF080430022DA607047000073
:103750004FF08043586370474FF08043586A70477A
:103760004B6843608B688360CB68C3600B694361BF
:103770004B6903628B6943620B680360704700000A
:1037800008B52C4B40F2FF712B481A690A431A61A5
:103790001A6922F4FF6222F007021A611A691A6B91
:1037A0000A431A631A6D0A431A65244A1B6D1146AF
:1037B000FFF7D6FF00F5806002F11C01FFF7D0FF94
:1037C00000F5806002F13801FFF7CAFF00F5806064
:1037D00002F15401FFF7C4FF00F5806002F17001AF
:1037E000FFF7BEFF00F5806002F18C01FFF7B8FF24
:1037F00000F5806002F1A801FFF7B2FF00F58060DC
:1038000002F1C401FFF7ACFF00F5806002F1E001B6
:10381000FFF7A6FF00F5806002F1FC01FFF7A0FFB3
:1038200002F58C7100F58060FFF79AFFBDE8084053
:1038300000F08AB80038024000000240383F00081B
:1038400008B500F02DFAFEF703FCFFF731F8BDE8EC
:103850000840FEF70BBE0000704700000F4B1A6CCB
:1038600042F001021A641A6E42F001021A660C4A12
:103870001B6E936843F0010393604FF080436B220B
:103880009A624FF0FF32DA6200229A615A63DA607C
:103890005A6001225A611A60704700BF0038024026
:1038A000002004E04FF0804208B51169D3680B4056
:1038B000D9B29B076FEA0101116107D5202383F379
:1038C0001188FEF7E5FB002383F3118808BD000093
:1038D0001B4B4FF0FF3000211A696FEA42526FEA2A
:1038E00052521A611A69C2F30A021A611A695A69B4
:1038F00058615A6959615A691A6A62F080521A62AB
:103900001A6A02F080521A621A6A5A6A58625A6A2D
:1039100059625A6A0B4A106840F480701060186F40
:1039200000F44070B0F5007F03D04FF4803018678A
:103930001967536823F40073536000F07DB900BF2A
:103940000038024000700040364B4FF44041364A88
:103950001A64364A11601A6842F001021A601A6845
:103960009207FCD59A6822F003029A602D4B9A6860
:1039700012F00C02FBD1196801F0F90119609A608C
:103980001A6842F480321A601A689003FCD55A6FA4
:1039900042F001025A67234B5A6F9107FCD5244A23
:1039A0005A601A6842F080721A60204B5A685204BA
:1039B000FCD51A6842F480321A605A68D003FCD5EC
:1039C0001A6842F400321A60184A53689903FCD509
:1039D000144B1A689201FCD5164A9A6040F2011203
:1039E000C3F88C200022C3F8902040F20733124A1B
:1039F0001360136803F00F03072BFAD1094B9A6881
:103A000042F002029A609A6802F00C02082AFAD187
:103A10005A6C42F480425A645A6E42F480425A66AA
:103A20005B6E7047003802400004001000700040D8
:103A30000836400900948838003C0240074A08B51F
:103A4000536903F00103536123B1054A13680BB1B5
:103A500050689847BDE80840FEF776BF003C01403B
:103A60003C3B0220074A08B5536903F00203536147
:103A700023B1054A93680BB1D0689847BDE8084068
:103A8000FEF762BF003C01403C3B0220074A08B5FC
:103A9000536903F00403536123B1054A13690BB161
:103AA00050699847BDE80840FEF74EBF003C014012
:103AB0003C3B0220074A08B5536903F008035361F1
:103AC00023B1054A93690BB1D0699847BDE8084016
:103AD000FEF73ABF003C01403C3B0220074A08B5D4
:103AE000536903F01003536123B1054A136A0BB104
:103AF000506A9847BDE80840FEF726BF003C0140E9
:103B00003C3B0220164B10B55C6904F478725A6194
:103B1000A30604D5134A936A0BB1D06A984760068E
:103B200004D5104A136B0BB1506B9847210604D58E
:103B30000C4A936B0BB1D06B9847E20504D5094A48
:103B4000136C0BB1506C9847A30504D5054A936CD0
:103B50000BB1D06C9847BDE81040FEF7F5BE00BF32
:103B6000003C01403C3B0220194B10B55C6904F459
:103B70007C425A61620504D5164A136D0BB1506D33
:103B80009847230504D5134A936D0BB1D06D984720
:103B9000E00404D50F4A136E0BB1506E9847A10490
:103BA00004D50C4A936E0BB1D06E9847620404D5CD
:103BB000084A136F0BB1506F9847230404D5054A88
:103BC000936F0BB1D06F9847BDE81040FEF7BCBEB5
:103BD000003C01403C3B022008B50348FDF714FBC4
:103BE000BDE80840FEF7B0BED423022008B5034864
:103BF000FDF70AFBBDE80840FEF7A6BE4024022000
:103C000008B50348FDF700FBBDE80840FEF79CBE81
:103C1000AC24022008B50348FDF7F6FABDE80840D9
:103C2000FEF792BE1825022008B5FFF73BFEBDE85F
:103C30000840FEF789BE0000062108B50846FFF7D8
:103C400097FB06210720FFF793FB06210820FFF7CB
:103C50008FFB06210920FFF78BFB06210A20FFF7C7
:103C600087FB06211720FFF783FB06212820FFF79B
:103C70007FFB07211C20FFF77BFB0C212620FFF791
:103C800077FB0C212720FFF773FB0C213520FFF772
:103C90006FFB0C215220BDE80840FFF769BB000014
:103CA00008B5FFF715FE00F00DF8FDF7BFFCFDF7B6
:103CB0008FFEFDF767FDFFF7CFFDBDE80840FFF77A
:103CC00037BD00000023054A19460133102BC2E915
:103CD000001102F10802F8D1704700BF3C3B0220FE
:103CE000034611F8012B03F8012B002AF9D1704784
:103CF00053544D3332463F3F3F3F3F3F0053544DB7
:103D0000333246375B347C355D780053544D333263
:103D100046375B367C375D7800000000402F02207C
:103D200018250220AC240220D423022040240220A3
:103D300000960000000000000000000000000000ED
:103D4000000000000000000000000000F515000861
:103D5000E11500081D1600080916000815160008D0
:103D600001160008ED150008D915000829160008ED
:103D70000000000001170008ED16000829170008D0
:103D800015170008211700080D170008F91600087C
:103D9000E5160008351700080000000001000000CB
:103DA000000000006D61696E0000000069646C65D0
:103DB00000000000AC3D0008C82D0220402F02206A
:103DC000010000004D20000800000000486F6C79E1
:103DD00062726F0025424F415244252D424C00250E
:103DE00053455249414C25000200000000000000EC
:103DF0001D1900088919000840004000E83702201A
:103E0000F83702200200000000000000030000005C
:103E100000000000CD1900080000000010000000A4
:103E2000083802200000000001000000000000002F
:103E3000AC3A0220010102000924000819230008FD
:103E4000B52300089923000843000000503E0008F5
:103E500009024300020100C032090400000102020D
:103E600001000524001001052401000104240202C0
:103E70000524060001070582030800FF090401006C
:103E8000020A000000070501024000000705810248
:103E900040000000120000009C3E000812011001CA
:103EA00002000040623151000002010203010000E3
:103EB0000403090425424F415244250050697868A3
:103EC00061776B3558003031323334353637383915
:103ED000414243444546000000800000008000004D
:103EE00000800000008000000000020000000400CC
:103EF00000000400000004000000040000000400B2
:103F0000000004000000040000000000151B000871
:103F1000CD1D0008791E000840004000243B02200F
:103F2000243B022001000000343B022080000000FE
:103F300040010000050000008000806A00020000CF
:103F4000AAAAAAAA40000040FFFF000000700000DB
:103F500000A00A000000080000000000AAAAAAAA07
:103F600000000400FFFF00000000000070000000DF
:103F70000000000100000000AAAAAAAA0000000098
:103F8000FFFF0000000000000000000020080A0001
:103F900000000000AAAAAAAA10040500FFFF000062
:103FA00000087000770000004004020028000000B4
:103FB000AAAAAAAA00000100FFFF0000000000005A
:103FC000080000000020000100000000AAAAAAAA20
:103FD00000100000FFFF00000000000800000000CB
:103FE0000041000000000000AAAAAAAA00400000A8
:103FF000FFFF00000000000000000000000400407F
:1040000000000000AAAAAAAA00040040FFFF0000C6
:10401000000000000000000000011500000000008A
:10402000AAAAAAAA00011500FFFF000000000000D4
:104030000000000000000000000000000000000080
:104040000000000000000000000000000000000070
:104050000000000000000000000000000000000060
:104060000000000000000000000000000000000050
:10407000330000000000000000801F00000000006E
:10408000FF00000000000000F03C00083F000000BE
:1040900049040000FD3C00083F00000051040000FE
:1040A0000B3D00083F0000000096000000000800E3
:1040B000960000000008000004000000B03E000868
:1040C00000000000000000000000000000000000F0
:0840D0000000000000000000E8
:00000001FF
